:10000000831600308500860083120030850086004C
:10001000FF308600A72091207430742000307420B7
:100020003130742002307420053074200830742080
:10003000303074200C30742006307420023074206C
:100040008820912074307420803074204C307420CB
:100050004030742000307420183074200030742038
:100060000030742000307420003074200030742080
:100070000030742000307420003074200030742070
:10008000003074200F3074201030742088209120AC
:1000900074307420003074203030742001307420AB
:1000A0000F307420882091207430742080307420A8
:1000B0008C30742040307420C8307420E5307420B7
:1000C000EC307420EC307420EF3074202030742039
:1000D000D7307420EF307420F2307420EC3074206C
:1000E000E4307420882073288F009E2008308E0012
:1000F0008510A7208F1B05148F1F0510A7208514BE
:10010000A7208510A7208F0D8E0B7828992000340A
:100110000510A7208514A7200514A7208510A72067
:10012000003405148514A7200510A7208510A720EA
:1001300000348514A7208510A7200034B02000309B
:1001400086000F088600B02000308600003408309A
:100150008C00FF308D008D0BAB288C0BA928003450
:1001600003308E00FF308C00FF308D008D0BB628E1
:0A0170008C0BB4288E0BB22800346B
:02400E00F93F78
:00000001FF
